:100000000C94F3000C940E010C940E010C940E0150
:100010000C940E010C940E010C942F160C940E01EE
:100020000C940E010C940E010C94FC150C94BD154F
:100030000C94C1100C940E010C940E010C940E0142
:100040000C940E010C9431040C940E010C94820F4C
:100050000C94D50F0C940E010C940E010C940E010F
:100060000C940E010C940E010C940E010C940E01D4
:100070004570692D4F5344205665722E302E382E10
:10008000322E330000416B7475656C6C65732053C0
:10009000657474696E67000053657474696E6720D7
:1000A000200000486F6568656E73656E736F72201F
:1000B00000004853206D697420536368616C746557
:1000C0007220000048656164696E6720486F6C6447
:1000D0002000004B6F6D706173732000004B6F6DDB
:1000E0007061737320666978200000475053204187
:1000F0006B74697620000041636873656E6B6F7086
:1001000070656C756E67200000447265687261747A
:100110006520626567722E2000004665686C657216
:100120002046433C2D3E4F5344200000556E7465DD
:10013000727370616E6E756E672000004B65696E3C
:10014000652053657474696E672D416E7A656967C1
:1001500065000050432F4254206973742065696E16
:100160006765736368616C746574000055656265EA
:10017000726E65686D65204C65747A746573205382
:10018000657474696E6700004F4E00002D2D2D00C0
:10019000004550492D4D656E750050616C0050430F
:1001A0002F4254004B656E6E756E670052432D42B0
:1001B000657472696562000045786974004F4E008D
:1001C0002D2D0076767D76767A76767E76767776C3
:1001D000767B76767876767C76767976767D7676A8
:1001E0007A76767E760011241FBECFEFD4E0DEBF94
:1001F000CDBF11E0A0E0B1E0ECEAFFE202C0059063
:100200000D92AC34B107D9F713E0ACE4B1E001C012
:100210001D92A039B107E1F70C941B010C9400006A
:1002200080E981BB8FE084BBAC9AAD9A8EE28ABB39
:10023000D99ADD9A08951F931092930110928F011D
:1002400010929401A0E0B0E00E94C217802D99277F
:1002500080935301A1E0B0E00E94C217802D99273E
:1002600080930001A2E0B0E00E94C217802D992780
:1002700080935401A7E1B0E00E94C217802D992716
:1002800080936B01A8E1B0E00E94C217802D9927EE
:1002900080937E010E9462150E9410010E94210439
:1002A00080915301813019F40E946D0F02C00E94A9
:1002B0005D0F7894A89A0E94B7030E9492040E944E
:1002C00099080E94E1080E94250980914E01813021
:1002D000B1F410924E0180919301882351F48091E2
:1002E0005301882331F480916001813011F40E9420
:1002F00077100E94B4100E94B9100E945E13809182
:10030000520190919301813041F4992331F40E947C
:10031000EF0D0E94E9120E94451280915101813037
:1003200099F580919301882379F5AA9A0E946D0E20
:1003300080916B01882399F40E94F7070E94E706D9
:1003400080917E0180FF04C00E9434110E946B09DD
:1003500080917E0183FF17C00E94EF1614C0809128
:100360000201823044F00E94A1080E9434110E94D0
:100370006B090E94680A80910201833024F00E9478
:10038000F7070E94E706AA9880914C018130C1F5D9
:10039000809193018823A1F510924C0180916B010B
:1003A000882321F080910201833014F00E942509F6
:1003B0008091680190916901019690936901809301
:1003C00068018091680190916901CC9769F48091EE
:1003D0006601909167010196909367018093660191
:1003E00010926901109268010E94CA0A0E941309C2
:1003F00080915901813021F40E947E0B0E940A0DE8
:1004000010914D01113009F060CF80919301882344
:1004100009F05BCF10924D010E94A10880917E01EE
:1004200085FF02C00E94451280918401813019F03D
:10043000823059F406C00E94660982E080938401EC
:1004400004C00E9449091093840180916B0181309E
:1004500009F03BCF80919301882309F036CF80913A
:100460006A01813009F031CF10926A018091020156
:10047000813071F082301CF4882339F026CF82302D
:1004800081F0833009F021CF17C00E9466091DCF8B
:100490000E94490964E084E00E9463020E94930480
:1004A00014CF0E94490964E084E00E9463020E9424
:1004B00099080E94E10809CF0E94490964E084E09C
:1004C0000E946302FCCE482FD99827E030E0DB98E9
:1004D000000000000000000081E090E0022E02C059
:1004E000880F991F0A94E2F7842311F0DA9A01C069
:1004F000DA980000000000000000DB9A0000000015
:1005000000000000215030408FEF2F3F3807F9F6F0
:1005100027E030E0DB98000000000000000081E0F0
:1005200090E0022E02C0880F991F0A94E2F78623FA
:1005300011F0DA9A01C0DA98000000000000000013
:10054000DB9A0000000000000000215030408FEFD7
:100550002F3F3807F9F6DB98DA98D99A089564E0C6
:1005600084E00E9463026CE480E00E9463021092C7
:100570004E0180914E018823E1F36AE08CE60E94EF
:10058000630260E085E00E94630208951F93CF93A9
:10059000DF9380914C018823E1F310924C010E947B
:1005A000291010E00DC080915101813011F40E949A
:1005B0006D0E80914C01813019F410924C0111E0C4
:1005C00090917F0180E0112309F481E0992311F4D7
:1005D000882349F7C8E1D0E0882309F4B1C08091AD
:1005E000740380937E0180917E01DE01082E0E94BB
:1005F000CA1745E850E061E082E00E941E0D48E91C
:1006000050E062E082E00E941E0D43EA50E064E0A8
:1006100082E00E941E0D42EB50E065E082E00E9405
:100620001E0D44EC50E066E082E00E941E0D43ED9A
:1006300050E067E082E00E941E0D4DED50E068E062
:1006400082E00E941E0D4BEE50E069E082E00E94C5
:100650001E0D47EF50E06AE082E00E941E0D4CE262
:1006600051E06BE082E00E941E0D40917C015091B0
:100670007D0162E084E10E94DF0C80917E0180FFB9
:1006800003C048E851E002C04CE851E064E084E176
:100690000E941E0D80917E0181FF03C048E851E059
:1006A00002C04CE851E065E084E10E941E0D80919B
:1006B0007E0182FF03C048E851E002C04CE851E0EF
:1006C00066E084E10E941E0D80917E0183FF03C0DD
:1006D00048E851E002C04CE851E067E084E10E9444
:1006E0001E0D80917E0184FF03C048E851E002C0E6
:1006F0004CE851E068E084E10E941E0D80917E018B
:1007000085FF03C048E851E002C04CE851E069E0D1
:1007100084E10E941E0D80917E0186FF03C048E89F
:1007200051E002C04CE851E06AE084E10E941E0DF5
:100730004091840355276BE084E10E94DF0C13C0D5
:1007400045E850E062E082E00E941E0D4AE151E07F
:1007500065E082E00E941E0DDE010E94C217802D1E
:10076000992780937E01DF91CF911F9108950E9478
:10077000AF0210924C0180914C018823E1F340E7D5
:1007800050E062E087E00E941E0D0E9493041092E8
:100790004C0180914C018823E1F310924C0180912F
:1007A0004C018823E1F310924C0164E084E00E9444
:1007B00063026CE480E00E9463028091530188230D
:1007C00019F40E94C6021AC04CE351E062E082E0D4
:1007D0000E941E0D43E551E064E082E00E941E0D80
:1007E0004CE651E066E082E00E941E0DA8E1B0E018
:1007F0000E94C217802D992780937E0180914C0121
:100800008823E1F310924C0180914C018823E1F39D
:1008100010924C0180914C018823E1F310924C011D
:1008200080914C018823E1F310924C0180914C019E
:100830008823E1F310924C0164E084E00E9463029B
:10084000089582E083BF92E49EBD8EE189BF83E07C
:1008500087BD86E982BD90938A0080E280937D0007
:1008600008951F920F920FB60F9211248F939F93AA
:10087000809150018F5F80935001809150018834A6
:1008800039F591E090934F011092500180918803C7
:100890008F5F8093880380918803843631F41092AF
:1008A000880390934C0190934D018091880382338B
:1008B00011F490934D01809187038F5F809387039C
:1008C000809187038A3021F41092870390934E0120
:1008D0009F918F910F900FBE0F901F901895282F0A
:1008E00080538A3010F090E005C0203311F49AE074
:1008F00001C0982F822F81548A3110F4922F965381
:10090000822F81568A3110F4922F9C532D3211F48C
:1009100099E403C02E3209F491E4892F992787FDC9
:1009200090950895089560E085E00E94630263E871
:1009300086E00E94630260E987E00E94630260E053
:1009400085E00E94630264E886E00E94630261E938
:1009500087E00E94630260E085E00E94630265E830
:1009600086E00E94630262E987E00E94630260E021
:1009700085E00E94630266E886E00E94630263E904
:1009800087E00E94630260E085E00E94630267E8FE
:1009900086E00E94630264E987E00E94630260E0EF
:1009A00085E00E94630268E886E00E94630265E9D0
:1009B00087E00E94630260E085E00E94630269E8CC
:1009C00086E00E94630266E987E00E94630260E0BD
:1009D00085E00E9463026AE886E00E94630267E99C
:1009E00087E00E94630260E085E00E94630261EAA2
:1009F00086E00E94630268E987E00E94630260E08B
:100A000085E00E94630262EA86E00E94630269E96F
:100A100087E00E94630260E085E00E94630263EA6F
:100A200086E00E9463026AE987E00E94630260E058
:100A300085E00E94630264EA86E00E9463026BE93B
:100A400087E00E94630260E085E00E94630265EA3D
:100A500086E00E9463026CE987E00E94630260E026
:100A600085E00E94630266EA86E00E9463026DE907
:100A700087E00E94630260E085E00E94630267EA0B
:100A800086E00E9463026EE987E00E94630260E0F4
:100A900085E00E94630268EA86E00E9463026FE9D3
:100AA00087E00E94630260E085E00E9463026FEBD2
:100AB00086E00E94630260EA87E00E94630260E0D1
:100AC00085E00E94630260EC86E00E94630261EAB6
:100AD00087E00E94630260E085E00E94630261ECAF
:100AE00086E00E94630262EA87E00E94630260E09F
:100AF00085E00E94630262EC86E00E94630263EA82
:100B000087E00E94630260E085E00E94630263EC7C
:100B100086E00E94630264EA87E00E94630260E06C
:100B200085E00E94630264EC86E00E94630265EA4D
:100B300087E00E94630260E085E00E94630265EC4A
:100B400086E00E94630266EA87E00E94630260E03A
:100B500085E00E94630266EC86E00E94630267EA19
:100B600087E00E94630260E085E00E9463026DED11
:100B700086E00E94630268EA87E00E94630260E008
:100B800085E00E9463026EED86E00E94630269EADE
:100B900087E00E94630260E085E00E9463026FEDDF
:100BA00086E00E9463026AEA87E00E94630260E0D6
:100BB00085E00E94630260EE86E00E9463026BEAB9
:100BC00087E00E94630260E085E00E94630261EEBC
:100BD00086E00E9463026CEA87E00E94630260E0A4
:100BE00085E00E94630262EE86E00E9463026DEA85
:100BF00087E00E94630260E085E00E94630263EE8A
:100C000086E00E9463026EEA87E00E94630260E071
:100C100085E00E94630264EE86E00E9463026FEA50
:100C200087E00E94630260E085E00E9463026BEF50
:100C300086E00E94630260EB87E00E94630260E04E
:100C400085E00E9463026CEF86E00E94630261EB24
:100C500087E00E94630260E085E00E9463026DEF1E
:100C600086E00E94630262EB87E00E94630260E01C
:100C700085E00E9463026EEF86E00E94630263EBF0
:100C800087E00E94630260E085E00E9463026FEFEC
:100C900086E00E94630264EB87E00E94630261E0E9
:100CA00085E00E94630260E086E00E94630265EBDB
:100CB00087E00E94630261E085E00E94630261E0D8
:100CC00086E00E94630266EB87E00E94630208955B
:100CD000FF920F931F93CF93DF938C01F62EEC01BD
:100CE00017C06D2F772785E00E9463026C2F86E086
:100CF0000E9463028F2D9927FC01EE0FFF1FE80F62
:100D0000F91FE15FFE4F608187E00E946302219638
:100D1000C8010596C817D90720F3E8012A9617C01D
:100D20006D2F772785E00E9463026C2F86E00E947A
:100D300063028F2D9927FC01EE0FFF1FE80FF91FAB
:100D4000E15FFE4F608187E00E9463022196C80147
:100D50000F96C817D90720F3DF91CF911F910F91FC
:100D6000FF9008950F931F93CF93DF938C01EC01B5
:100D70000EC06D2F772785E00E9463026C2F86E0FE
:100D80000E94630260E087E00E9463022196C8012E
:100D90000596C817D90768F3E8012A960EC06D2F8B
:100DA000772785E00E9463026C2F86E00E94630231
:100DB00060E087E00E9463022196C8010F96C81781
:100DC000D90768F3DF91CF911F910F9108951F9379
:100DD000CF93DF93809128039091290366E170E01F
:100DE0000E948D179B012E5F3F4F37FD1BC0C9012D
:100DF0006AE070E00E948D17182F1695C9016AE00D
:100E000070E00E948D1787E090E0861B91092EE12B
:100E100030E0829FE001839FD00D929FD00D11247E
:100E2000279616C0309521953F4FC9016AE070E0C2
:100E30000E948D17182F16951C5FC9016AE070E09B
:100E40000E948D178EE1689FE0011124C950DF4F89
:100E500080910B0190910C01C817D90739F080914E
:100E60000B0190910C010E94B20604C08091820196
:100E7000811721F0612FCE010E9468061093820134
:100E8000D0930C01C0930B01DF91CF911F91089576
:100E9000AF92BF92DF92EF92FF920F931F93CF9387
:100EA000DF93CDB7DEB721970FB6F894DEBF0FBE44
:100EB000CDBF8C01D62E5C0119826B2D772785E082
:100EC0000E9463026A2D86E00E946302ED2CFF24DB
:100ED000F701E35DFE4F608187E00E9463028EE1CF
:100EE00090E0A80EB91E9981925E99839C3329F7F0
:100EF000F4EBAF2EB12CA00EB11E6B2D772785E041
:100F00000E9463026A2D86E00E946302F701E35D9E
:100F1000FE4F608187E00E946302EEE1F0E0AE0EDA
:100F2000BF1EC801825F9E4FA816B90631F72196F1
:100F30000FB6F894DEBF0FBECDBFDF91CF911F91EA
:100F40000F91FF90EF90DF90BF90AF900895EF92D8
:100F5000FF920F931F93CF93DF93CDB7DEB7219707
:100F60000FB6F894DEBF0FBECDBF8C017C01198295
:100F70006F2D772785E00E9463026E2D86E00E9428
:100F8000630260E087E00E9463028EE190E0E80E79
:100F9000F91E9981925E99839C3351F784EBE82E78
:100FA000F12CE00EF11E6F2D772785E00E94630281
:100FB0006E2D86E00E94630260E087E00E9463027B
:100FC000EEE1F0E0EE0EFF1EC801825F9E4FE816D4
:100FD000F90649F721960FB6F894DEBF0FBECDBFD4
:100FE000DF91CF911F910F91FF90EF9008951F9384
:100FF000CF93DF9380912A0390912B0366E170E0F9
:101000000E948D179B012A5F3F4F37FD12C0C90117
:101010006AE070E00E948D17182F16951C5FC901B9
:101020006AE070E00E948D17C6E8D0E0C61BD109C7
:1010300013C0309521953F4FC9016AE070E00E94CE
:101040008D17182F1695C9016AE070E00E948D1760
:10105000C62FDD27C957DF4F80910D0190910E01FA
:10106000C817D90739F080910D0190910E010E94A7
:10107000A70704C080918301811721F0612FCE0161
:101080000E94480710938301D0930E01C0930D0175
:10109000DF91CF911F91089560E085E00E94630287
:1010A0006FEC86E00E9463026CE887E00E946302B6
:1010B00061E085E00E9463026BE086E00E946302CB
:1010C0006DE887E00E9463020895EF92FF920F930C
:1010D0001F93CF93DF937A019EE1699FB0011124A2
:1010E000680F711D8B01020F111D10928903EB0116
:1010F00016C06D2F772785E00E9463026C2F86E073
:101100000E94630280918903F701E80FF11D60815D
:101110008F5F8093890387E00E9463022196C01746
:10112000D10738F3DF91CF911F910F91FF90EF908E
:10113000089525E046E051E06EE081E00E946508F8
:101140000895CF93DF93CDB7DEB724970FB6F89409
:10115000DEBF0FBECDBF19821A8285E48B831C824D
:10116000F894789430913A03832F6AE00E946D17C7
:10117000282F0E946D17482F822F0E946D17292F4C
:10118000832F0E946D17992319F48AE08C8301C084
:101190009C83222319F48AE08A8301C02A8349832D
:1011A00024E0AE014F5F5F4F61E083E00E9465087D
:1011B00024960FB6F894DEBF0FBECDBFDF91CF915E
:1011C0000895CF93DF93CDB7DEB724970FB6F89489
:1011D000DEBF0FBECDBF80E28A839BE0998381E3AF
:1011E0008B839C8321E0AE014E5F5F4F61E081E025
:1011F0000E94650821E0AE014F5F5F4F62E081E031
:101200000E94650822E0AE014D5F5F4F63E081E020
:101210000E94650824960FB6F894DEBF0FBECDBFBE
:10122000DF91CF91089580915401813069F420912C
:10123000A101922F27FD9F5F959542EA51E061E061
:101240008EE0891B0E9465080895CF93DF93CDB788
:10125000DEB725970FB6F894DEBF0FBECDBFDE0117
:101260001196EAE3F1E085E001900D928150E1F7FB
:1012700025E0AE014F5F5F4F67E08CE00E9465089C
:1012800025960FB6F894DEBF0FBECDBFDF91CF918C
:1012900008956CE480E00E946302089580913C030D
:1012A00090913D03843B910544F48091840188230F
:1012B00061F481E08093840108958091840118167F
:1012C00014F40E94490910928401089562E480E0B8
:1012D0000E9463020895EF92FF920F931F93CF93A2
:1012E000DF93CDB7DEB72F970FB6F894DEBF0FBEF2
:1012F000CDBF85E0FE01369611928A95E9F780917F
:101300003203909133036EE170E00E948D17CB01A0
:101310008E01055F1F4F019797FF02C080E090E0AC
:101320004AE050E0B8010E943C17F801019000200B
:10133000E9F73197EE2EE01A10928903FF240AC0D4
:101340000E0F1F1FEC0FFD1F83850E946F04F80115
:101350008083F394EF2DFF278E2D992787FD90959D
:101360008E010F5F1F4FE817F90754F3F0928903BE
:1013700025E0AE014A5F5F4F69E085E10E946508A4
:101380002E2DA80169E089E18E190E9465082F962B
:101390000FB6F894DEBF0FBECDBFDF91CF911F9186
:1013A0000F91FF90EF900895EF92FF920F931F938C
:1013B000CF93DF93CDB7DEB72E970FB6F894DEBF8D
:1013C0000FBECDBF19821A821B821C8280917401CC
:1013D000909175018E01065F1F4F4AE050E0B80101
:1013E0000E943C17F80101900020E9F73197EE2E9A
:1013F000E01A10928903FF240AC00E0F1F1FEC0F82
:10140000FD1F82850E946F04F8018083F394EF2D05
:10141000FF278E2D992787FD90958E010B5F1F4F1B
:10142000E817F90754F3F092890324E0AE014F5F07
:101430005F4F66E085E10E9465082E2DA80166E0F9
:1014400089E18E190E94650880917401909175015F
:101450001816190664F460E085E00E94630262ECED
:1014600086E00E9463026CE887E00E94630280913C
:1014700074019091750197FF0CC060E085E00E94B7
:10148000630262EC86E00E9463026DE887E00E94DE
:1014900063028091740190917501892B61F460E081
:1014A00085E00E94630262EC86E00E94630260E0D5
:1014B00087E00E9463022E960FB6F894DEBF0FBE3F
:1014C000CDBFDF91CF911F910F91FF90EF900895C5
:1014D000EF92FF920F931F93CF93DF93CDB7DEB7B9
:1014E0002B970FB6F894DEBF0FBECDBFDE0111966D
:1014F000E7E3F1E083E001900D928150E1F78E0186
:10150000085F1F4F4AE050E0B80180913803909186
:1015100039030E943C17F80101900020E9F7319748
:10152000EE2EE01A10928903FF240AC00E0F1F1F2F
:10153000EC0FFD1F80850E946F04F8018083F394F7
:10154000EF2DFF278E2D992787FD90958E010C5F3B
:101550001F4FE817F90754F3F092890323E0AE0117
:101560004F5F5F4F6EE08DE00E9465082E2DA80151
:101570006EE080E18E190E9465082B960FB6F894F4
:10158000DEBF0FBECDBFDF91CF911F910F91FF90B6
:10159000EF900895EF92FF920F931F93CF93DF93F5
:1015A000CDB7DEB728970FB6F894DEBF0FBECDBF1C
:1015B00019828AE08A8380916601909167018E0189
:1015C0000A5F1F4F4AE050E0B8010E943C17F80143
:1015D00001900020E9F73197EE2EE01A109289036E
:1015E000FF240DC08E010D5F1F4F0E0F1F1FEC0F4C
:1015F000FD1F86810E946F04F8018083F394EF2D14
:10160000FF278E2D992787FD9095E817F90754F34A
:10161000F092890380916601909167018E010D5FC0
:101620001F4F0A976CF421E0AE014F5F5F4F6EE0F1
:1016300081E00E94650821E0A8016EE082E004C01C
:1016400022E0A8016EE081E00E94650880916801B7
:10165000909169018E010A5F1F4F4AE050E0B80186
:101660000E943C17F80101900020E9F73197EE2E17
:10167000E01A10928903FF240DC08E010D5F1F4FE9
:101680000E0F1F1FEC0FFD1F86810E946F04F801D3
:101690008083F394EF2DFF278E2D992787FD90955A
:1016A000E817F90754F3F09289038091680190914B
:1016B00069018E010D5F1F4F0A976CF421E0AE01A6
:1016C0004E5F5F4F6EE084E00E94650821E0A80154
:1016D0006EE085E004C022E0A8016EE084E00E9494
:1016E000650828960FB6F894DEBF0FBECDBFDF9118
:1016F000CF911F910F91FF90EF900895CF92DF92BD
:10170000EF92FF920F931F93CF93DF93CDB7DEB786
:101710002B970FB6F894DEBF0FBECDBF80915A0154
:1017200090915B0180915A0190915B018D5A964294
:1017300030F08CEA96E290935B0180935A0180919D
:101740005A0190915B0164E670E00E9479177093F2
:1017500056016093550180915A0190915B0164E6B6
:1017600070E00E94791790935801809357018091FF
:101770005701909158016AE070E00E9479177093C8
:10178000580160935701809155019091560125E4CD
:1017900029831A821B828E01085F1F4F4AE050E0A6
:1017A000B8010E943C17F80101900020E9F7319739
:1017B000CE2EC01A10928903DD240BC0020F131F16
:1017C000E20EF31EF70180810E946F04F80180830E
:1017D000D3942D2D33278C2D992787FD909548E0A4
:1017E000E42EF12CEC0EFD1E8E010C5F1F4F28170E
:1017F000390724F3D092890322E0AE014E5F5F4F98
:1018000062E083E00E9465082C2DA80162E085E07B
:101810008C190E94650880915701909158014AE007
:1018200050E0B7010E943C17F70101900020E9F752
:101830003197EE19EE2E10928903FF240AC00E0F85
:101840001F1FEC0FFD1F80850E946F04F80180832D
:10185000F394EF2DFF278E2D992787FD90958E010C
:101860000C5F1F4FE817F90754F3F092890321E04A
:10187000AE014F5F5F4F62E085E00E94650821E0A6
:10188000AE014E5F5F4F62E086E00E94650821E096
:10189000A80162E086E00E9465082B960FB6F894D6
:1018A000DEBF0FBECDBFDF91CF911F910F91FF9093
:1018B000EF90DF90CF9008950F931F93CF93DF9316
:1018C000CDB7DEB72A970FB6F894DEBF0FBECDBFF7
:1018D0004AE050E08E010F5F1F4FB8010E943C1795
:1018E000F80101900020E9F73197E01B109289037D
:1018F00020E0FF27E7FDF09501C02F5F822F992799
:101900008E179F07D4F3209389032A960FB6F89475
:10191000DEBF0FBECDBFDF91CF911F910F91089514
:101920009F92AF92BF92CF92DF92EF92FF920F936E
:101930001F93CF93DF93CDB7DEB76E970FB6F894B2
:10194000DEBF0FBECDBF982EA62E7A01FA01019000
:101950000020E9F73197BE2EB41ACC24DD240BC049
:10196000FF278A010E0F1F1FEE0DFF1D80810E94B1
:101970006F04F8018083EC2D0894C11CD11C8B2DC1
:1019800099270196AE014F5F5F4FC816D90641F700
:101990002B2D6A2D892D0E9465086E960FB6F8943E
:1019A000DEBF0FBECDBFDF91CF911F910F91FF9092
:1019B000EF90DF90CF90BF90AF909F900895EF92FF
:1019C000FF920F931F93CF93DF93CDB7DEB764974A
:1019D0000FB6F894DEBF0FBECDBFE82EF62ECA01BB
:1019E0004AE050E08E010F5F1F4FB8010E943C1784
:1019F000A8016F2D8E2D0E94900C64960FB6F8945E
:101A0000DEBF0FBECDBFDF91CF911F910F91FF9031
:101A1000EF90089560915C0170915D0180915E018D
:101A200090915F0128E631E040E050E00E94A0176D
:101A3000A90163E083E00E94DF0C0895BF92CF927A
:101A4000DF92EF92FF920F931F93CF93DF93CDB767
:101A5000DEB764970FB6F894DEBF0FBECDBFB82EC9
:101A6000C62E9A01DE01119605C0EA0FFB1F908376
:101A70002F5F3F4F822F841BF9019491E82FFF279E
:101A8000992399F7EA0FFB1F1082FD0101900020B6
:101A9000E9F73197DE2EDA1AEE24FF2409C08D0112
:101AA000020F111DF80180810E946F04F8018083EC
:101AB0002E2D0894E11CF11C8D2D99270196DE0135
:101AC0001196E816F90659F72D2DAD016C2D8B2DC9
:101AD0000E94650864960FB6F894DEBF0FBECDBFB6
:101AE000DF91CF911F910F91FF90EF90DF90CF90FA
:101AF000BF9008950F931F93CF93DF9360E070E042
:101B0000C3E0D0E0A3E9B2E03C91FD012181128164
:101B10000381CE010496EC011496835D924009F492
:101B200059C0422F55274D535040E0914301F09149
:101B30004401E60FF71F832F9927CD97880F991F30
:101B4000880F991F9A01689413F835952795169474
:101B5000E1F7822B932B808368317105D9F1212F16
:101B600033272D533040FB013196809143019091F2
:101B70004401E80FF91F4F70507084E0440F551F67
:101B80008A95E1F7C9019595879595958795482B95
:101B9000592B408381E067317807E1F0FB013296F1
:101BA0008091430190914401E80FF91F2370307038
:101BB00086E0220F331F8A95E1F7802F9927CD9772
:101BC000282B392B2083E2E066317E0719F06D5F08
:101BD0007F4F9ACFDF91CF911F910F910895EF9290
:101BE000FF920F931F93CF93DF938091B8018434BA
:101BF00009F06AC033E0E32EF12C60E070E0A9EB5D
:101C0000B1E08C91FD01218112810381E7012496CD
:101C10007E0114966134710509F456C0422F552790
:101C20004D535040E0914101F0914201E60FF71F02
:101C30009927CD97880F991F880F991F9A0168944B
:101C400013F8359527951694E1F7822B932B808313
:101C500060347105C9F1212F33272D533040FB012A
:101C600031968091410190914201E80FF91F4F7028
:101C7000507084E0440F551F8A95E1F7C90195958E
:101C8000879595958795482B592B4083CB35D10562
:101C9000D9F0FB0132968091410190914201E80F09
:101CA000F91F2370307046E0220F331F4A95E1F789
:101CB000802F9927CD97282B392B20836E337105E0
:101CC00019F06D5F7F4F9DCF10925201DF91CF9140
:101CD0001F910F91FF90EF900895EF92FF920F9355
:101CE0001F93CF93DF9380919202843409F091C0C7
:101CF00033E0E32EF12C60E070E0A3E9B2E08C91D8
:101D0000FD01218112810381E70124967E01149651
:101D10006134710509F456C0422F55274D53504088
:101D2000E0913F01F0914001E60FF71F9927CD9711
:101D3000880F991F880F991F9A01689413F8359599
:101D400027951694E1F7822B932B808360347105DD
:101D5000C9F1212F33272D533040FB01319680915B
:101D60003F0190914001E80FF91F4F70507084E0DF
:101D7000440F551F8A95E1F7C9019595879595956B
:101D80008795482B592B4083CB35D105D9F0FB01E2
:101D9000329680913F0190914001E80FF91F237026
:101DA000307046E0220F331F4A95E1F7802F9927C4
:101DB000CD97282B392B20836E33710519F06D5F79
:101DC0007F4F9DCF80913C0390913D03843B9105D3
:101DD0008CF4809160018130E1F410926001F894FC
:101DE0000E946D0F789480913C0390913D03843B59
:101DF00091057CF080916001882359F481E0809303
:101E00006001F89480915301882311F40E945D0FC2
:101E10007894809192028C3459F481E090E0909310
:101E20007D0180937C0181E080937F010E947A0D87
:101E3000809192028D3459F482E090E090937D017C
:101E400080937C0181E080937F010E947A0D8091D4
:101E500092028E3459F483E090E090937D01809358
:101E60007C0181E080937F010E947A0D8091920233
:101E70008F3459F484E090E090937D0180937C014D
:101E800081E080937F010E947A0D809192028035DB
:101E900059F485E090E090937D0180937C0181E08E
:101EA00080937F010E947A0D10925101DF91CF91B2
:101EB0001F910F91FF90EF90089582E289B910BCB5
:101EC00080B91CBE909A28E92AB996E890BD82ECA8
:101ED0008BB921B99CBF82B9089582E289B910BC3F
:101EE00080B91CBE909A88E98AB926E820BD92EC98
:101EF0009BB980E981B92CBF92B90895159BFECF9B
:101F000083B908951F920F920FB60F9211248F93E9
:101F10009F93EF93FF939CB190938A039D3081F43C
:101F200080918601813061F4AB9810928601809394
:101F30005201E0916B03FF27EA54FE4F90832CC0BF
:101F400080918601882319F0813031F513C09332D6
:101F500039F480915201882319F481E0809386013D
:101F600010926B0380916B03E82FFF27EA54FE4F1A
:101F700090830CC0E0916B03FF27EA54FE4F9083DF
:101F800080916B03853930F480916B038F5F809370
:101F90006B0302C010928601FF91EF919F918F9188
:101FA0000F900FBE0F901F9018951F920F920FB6B3
:101FB0000F9211248F939F93EF93FF9393B190937C
:101FC0008B039D3081F480918501813061F4AB9861
:101FD0001092850180935101E0916803FF27E0573B
:101FE000FD4F90832DC080918501882319F08130A9
:101FF00039F514C0933241F480915101882321F4C2
:1020000081E080938501AB9A109268038091680308
:10201000E82FFF27E057FD4F90830CC0E091680345
:10202000FF27E057FD4F908380916803853930F496
:10203000809168038F5F8093680302C010928501CE
:10204000FF91EF919F918F910F900FBE0F901F9076
:102050001895CF93DF93CDB7DEB72C970FB6F894D2
:10206000DEBF0FBECDBF83E289831A8281E78B83F7
:102070008CE78C838DE68D838DE38E838F8320E0C8
:1020800030E0FE013196AE01485F5F4F8191280F2D
:10209000311DE417F507D1F7C90160E070E10E9436
:1020A0008D179C0160E470E00E948D17635C688767
:1020B000C90160E470E00E948D17835C89878DE020
:1020C0008A87FE0131969E01255F3F4F8081159BD7
:1020D000FECF83B93196E217F307C1F72C960FB6FE
:1020E000F894DEBF0FBECDBFDF91CF910895CF939F
:1020F000DF93CDB7DEB72A970FB6F894DEBF0FBED9
:10210000CDBF83E289831A8283E68B831C821D8282
:1021100086E890E060E070E10E948D179C0160E429
:1021200070E00E948D17635C6E83C90160E470E00B
:102130000E948D17835C8F838DE08887FE01319626
:102140009E01275F3F4F8081159BFECF83B931965B
:10215000E217F307C1F72A960FB6F894DEBF0FBE59
:10216000CDBFDF91CF91089585B392E0892785BBDC
:10217000089590916301913019F485B3892785BB47
:1021800008951F920F920FB60F9211242F933F9331
:102190005F936F937F938F939F93AF93BF93809140
:1021A000870190918801892B81F484B595B590932E
:1021B0008E0180938D018EB58F7B8EBD81E090E086
:1021C000909388018093870141C084B595B5909321
:1021D0008C0180938B012EB520642EBD20918D0142
:1021E00030918E01821B930B10928801109287010F
:1021F000865698406CE271E00E94791770938A01CC
:102200006093890177FF05C010928A0110928901BD
:1022100009C06730710534F086E090E090938A0140
:10222000809389012091890130918A018091020176
:10223000992787FD90952817390741F026303105F9
:102240002CF42093020181E080936A01BF91AF9149
:102250009F918F917F916F915F913F912F910F90FF
:102260000FBE0F901F901895809132039091330309
:1022700090936D0180936C0180916C0190916D0140
:1022800020916E0130916F01821B930B909371012D
:102290008093700180916C0190916D0190936F011A
:1022A00080936E01409178015091790120917001E5
:1022B00030917101CA01E3E0880F991FEA95E1F7B7
:1022C000841B950B73E0220F331F7A95E1F7820F81
:1022D000931F68E070E00E948D17709379016093FE
:1022E000780120917A0130917B01409178015091E1
:1022F0007901C90163E0880F991F6A95E1F7821B94
:10230000930B840F951F68E070E00E948D17709307
:102310007B0160937A0180917A0190917B01909387
:102320007501809374010E94D4090895BF92CF92E1
:10233000DF92EF92FF920F931F93CF93DF93CDB76E
:10234000DEB760970FB6F894DEBF0FBECDBF19821F
:102350001A821B821C828091840290918502909344
:102360008F0380938E0380918602909187029093D1
:102370008D0380938C0380918E0390918F038E0147
:10238000055F1F4F4AE050E0B8010E943C17F8017A
:1023900001900020E9F73197BE2EB01ACC24DD243D
:1023A0000DC0EC0CFD1CF70180810E946F040C0D28
:1023B0001D1DF80180830894C11CD11C8B2D992709
:1023C00087FD90952BE0E22EF12CEC0EFD1E8E0188
:1023D0000B5F1F4FC816D90624F324E0AE014F5FF0
:1023E0005F4F61E08CE00E9465082B2DA80161E041
:1023F00080E18B190E94650880918C0390918D0378
:102400004AE050E0B7010E943C17F701019000201C
:10241000E9F73197DE2EDE18EE24FF240DC0FE0111
:10242000EE0DFF1D83850E946F040E0D1F1DF80128
:1024300080830894E11CF11C8D2D992787FD9095D0
:102440008E010B5F1F4FE816F9064CF324E0AE0136
:102450004F5F5F4F62E08CE00E9465082D2DA80160
:1024600062E080E18D190E94650860960FB6F894CD
:10247000DEBF0FBECDBFDF91CF911F910F91FF90B7
:10248000EF90DF90CF90BF9008958F929F92BF9270
:10249000CF92DF92EF92FF920F931F93CF93DF9330
:1024A000CDB7DEB760970FB6F894DEBF0FBECDBFD5
:1024B00019821A821B821C8280904C0390904D03DB
:1024C0008E01055F1F4F4AE050E0B80180914A033A
:1024D00090914B030E943C17F80101900020E9F70E
:1024E0003197BE2EB01ACC24DD240DC0EC0CFD1C9F
:1024F000F70180810E946F040C0D1D1DF80180837F
:102500000894C11CD11C8B2D992787FD90953BE029
:10251000E32EF12CEC0EFD1E8E010B5F1F4FC81633
:10252000D90624F324E0AE014F5F5F4F6DE084E1F4
:102530000E9465082B2DA8016DE088E18B190E948F
:1025400065084AE050E0B701C4010E943C17F7015A
:1025500001900020E9F73197DE2EDE18EE24FF24EB
:102560000DC0FE01EE0DFF1D83850E946F040E0D50
:102570001F1DF80180830894E11CF11C8D2D992703
:1025800087FD90958E010B5F1F4FE816F9064CF3FF
:1025900024E0AE014F5F5F4F6EE084E10E9465086A
:1025A0002D2DA8016EE088E18D190E9465086096C6
:1025B0000FB6F894DEBF0FBECDBFDF91CF911F9154
:1025C0000F91FF90EF90DF90CF90BF909F908F90F2
:1025D0000895DF92EF92FF920F931F93CF93DF93B3
:1025E000CDB7DEB72B970FB6F894DEBF0FBECDBFC9
:1025F000DE011196E9E4F1E083E001900D92815053
:10260000E1F78E01085F1F4F4AE050E0B80180916A
:102610008C0290918D020E943C17F80101900020DD
:10262000E9F73197DE2ED01AEE24FF240DC0FE010B
:10263000EE0DFF1D80850E946F040E0D1F1DF80119
:1026400080830894E11CF11C8D2D992787FD9095BE
:102650008E010C5F1F4FE816F9064CF323E0AE0124
:102660004F5F5F4F61E088E10E9465082D2DA80152
:1026700061E08BE18D190E9465082B960FB6F894E6
:10268000DEBF0FBECDBFDF91CF911F910F91FF90A5
:10269000EF90DF90089522E047E451E061E08AE1A5
:1026A0000E9465080895F89488E190E028E00FB64C
:1026B000F894A89581BD0FBE21BDFFCF1F939D99B2
:1026C00002C180918F018F5F80938F0191E0909381
:1026D000910180918F01853009F0F9C080919301BB
:1026E000882309F071C0909393011092940164E0E3
:1026F00084E00E9463022091A10142EA51E061E07E
:1027000083E00E94650841E951E063E083E00E94B4
:102710001E0D68E084E00E9463024AE951E065E032
:1027200083E00E941E0D80910001813019F44DEB71
:1027300051E002C040EC51E065E084E10E941E0DD2
:1027400060E084E00E9463024EE951E066E083E0CD
:102750000E941E0D80915301813019F44DEB51E020
:1027600002C040EC51E066E084E10E941E0D44EAA4
:1027700051E067E083E00E941E0D8091540181309A
:1027800019F44DEB51E002C040EC51E067E084E108
:102790000E941E0D4CEA51E068E083E00E941E0D8D
:1027A00080916B01813019F44DEB51E002C040EC97
:1027B00051E068E084E10E941E0D48EB51E06BE0BF
:1027C00083E00E941E0D81C010919401113001F52B
:1027D00068E084E00E94630280915301882329F419
:1027E000109353014DEB51E004C01092530140ECA3
:1027F00051E066E084E10E941E0D80915301A0E04B
:10280000B0E0082E0E94CA1760E084E00E946302D4
:1028100080919401823009F568E084E00E946302AF
:1028200080915401882331F481E0809354014DEB71
:1028300051E004C01092540140EC51E067E084E1A3
:102840000E941E0D80915401A2E0B0E0082E0E946B
:10285000CA1760E084E00E94630280919401833093
:1028600009F568E084E00E94630280916B0188238F
:1028700031F481E080936B014DEB51E004C0109284
:102880006B0140EC51E068E084E10E941E0D8091F4
:102890006B01A7E1B0E0082E0E94CA1760E084E057
:1028A0000E94630280919401843089F41092930114
:1028B000F89488E190E028E00FB6F894A89581BDDF
:1028C0000FBE21BDFFCF10928F01109291019C99F4
:1028D000E9C090919301913009F0EAC09093920180
:1028E000809190018F5F809390018091900185305D
:1028F00009F0DEC01092900180919401823009F4B9
:1029000064C0833030F4882359F0813009F0D0C09E
:1029100031C0833009F483C0843009F0C9C09EC03F
:10292000909394014AE951E065E083E00E941E0D16
:1029300080910001813019F44DEB51E002C040EC70
:1029400051E065E084E10E941E0D68E084E00E9491
:1029500063024EE951E066E083E00E941E0D809123
:102960005301813019F44DEB51E002C040EC51E0CD
:1029700066E090C082E0809394014EE951E066E009
:1029800083E00E941E0D80915301813019F44DEBBC
:1029900051E002C040EC51E066E084E10E941E0D6F
:1029A00068E084E00E94630244EA51E067E083E06B
:1029B0000E941E0D80915401813019F44DEB51E0BD
:1029C00002C040EC51E067E065C083E08093940171
:1029D00044EA51E067E00E941E0D8091540181306D
:1029E00019F44DEB51E002C040EC51E067E084E1A6
:1029F0000E941E0D68E084E00E9463024CEA51E0F0
:102A000068E083E00E941E0D80916B01813019F413
:102A10004DEB51E002C040EC51E068E03BC084E087
:102A2000809394014CEA51E068E083E00E941E0D1F
:102A300080916B01813019F44DEB51E002C040EC04
:102A400051E068E084E10E941E0D68E084E00E948D
:102A5000630248EB51E06BE083E01DC010929401EB
:102A600048EB51E06BE083E00E941E0D68E084E0DB
:102A70000E9463024AE951E065E083E00E941E0D76
:102A800080910001813019F44DEB51E002C040EC1F
:102A900051E065E084E10E941E0D60E084E00E9448
:102AA000630206C010929001809191018091920181
:102AB0001F910895813029F4A0E0B0E0062E0E9415
:102AC000CA170895EF92FF920F931F93CF93DF934E
:102AD000CDB7DEB764970FB6F894DEBF0FBECDBF9B
:102AE00040E050E08E010F5F1F4F842F9927DC01DB
:102AF000AD5FBF4F0E94C217202D3327F801E80FAA
:102B0000F91F20832223F1F04F5F5F4F2F3F69F7BA
:102B1000108218C0FE01E00FF11F81810E946F0436
:102B20000E551E4FF80180830E2D11270894E11CCD
:102B3000F11C8091A101992787FD9095081719072D
:102B40004CF30EC0DE011196FD0101900020E9F763
:102B50003197EA1BFB0BE093A101EE24FF24E4CFA5
:102B600064960FB6F894DEBF0FBECDBFDF91CF9154
:102B70001F910F91FF90EF9008951F920F920FB643
:102B80000F9211248F939F93809198018130A1F02F
:102B9000813018F0823049F525C0809196018E3140
:102BA00029F41092960181E080939801809196011A
:102BB0008F5F8093960119C090919701923061F4D4
:102BC0001092970180919501813019F490939801AA
:102BD00003C083E080939801809197018F5F809379
:102BE000970103C083E0809398019F918F910F908C
:102BF0000FBE0F901F9018951F920F920FB60F9255
:102C000011248F9380919801833011F410929801D0
:102C10008F910F900FBE0F901F90189580912803F1
:102C20009091290365E070E00E948D1766507F4FF8
:102C300077FD0FC081E0653F78071CF064EF71E01D
:102C400003C06B3F71053CF06A5F81E080939501A2
:102C500004C060E070E01092950162BD08951F927B
:102C60000F920FB60F921124EF92FF920F931F93C2
:102C70002F933F934F935F936F937F938F939F9384
:102C8000AF93BF93EF93FF9321E02093590180917D
:102C90009901882381F48091800090918100909324
:102CA000A00180939F0180918A008F7B80938A008E
:102CB000209399017FC08091800090918100909332
:102CC0005B0180935A0180918A00806480938A001E
:102CD00010928900109288001092990180915A01F7
:102CE00090915B0120919F013091A001821B930B79
:102CF00090935B0180935A0180915A0190915B01FE
:102D00009695879590935B0180935A0180915A0123
:102D100090915B018456904090935B0180935A019F
:102D200080915A0190915B019C0144275527809125
:102D30009A0190919B01A0919C01B0919D01280F57
:102D4000391F4A1F5B1F20939A0130939B014093C8
:102D50009C0150939D0180919E01843130F110922D
:102D60009E01E0905C01F0905D0100915E01109188
:102D70005F01CA01B90124E130E040E050E00E9467
:102D8000A017E20EF31E041F151FE0925C01F092E3
:102D90005D0100935E0110935F0110929A01109201
:102DA0009B0110929C0110929D0180919E018F5F6A
:102DB00080939E01FF91EF91BF91AF919F918F9171
:102DC0007F916F915F914F913F912F911F910F9143
:102DD000FF90EF900F900FBE0F901F901895CF931C
:102DE000DF93CDB7DEB760970FB6F894DEBF0FBEA6
:102DF000CDBF809138039091390390938F028093D7
:102E00008E0280918E0290918F026FE070E00E949E
:102E10007917AE014B5F5F4FDA01641BCE0140961C
:102E2000E62FEA0FFF27ED53FE4FE491ED93A8172D
:102E3000B907B1F719821A821B821C822BE06EE05F
:102E400089E00E94650824E0AE014F5F5F4F6CE0AF
:102E50008EE00E94650840918E0250918F026CE0D6
:102E60008FE00E94DF0C60960FB6F894DEBF0FBEB5
:102E7000CDBFDF91CF910895FB019F01E8944230CF
:102E8000C4F04532B4F44A3029F497FB1EF490950F
:102E900081959F4F642F77270E947917805D8A3331
:102EA0000CF0895D8193CB010097A1F716F45DE2E8
:102EB00051931082C9010C945D17DC01FC01019053
:102EC0000020E9F73297AE17BF0730F47C9160819C
:102ED000708331976D93F7CF0895991B79E004C003
:102EE000991F961708F0961B881F7A95C9F7809549
:102EF0000895AA1BBB1B51E107C0AA1FBB1FA61741
:102F0000B70710F0A61BB70B881F991F5A95A9F792
:102F100080959095BC01CD01089597FB092E072659
:102F20000AD077FD04D0E5DF06D000201AF47095B2
:102F300061957F4F0895F6F7909581959F4F08957D
:102F4000A1E21A2EAA1BBB1BFD010DC0AA1FBB1FAD
:102F5000EE1FFF1FA217B307E407F50720F0A21B1F
:102F6000B30BE40BF50B661F771F881F991F1A948C
:102F700069F760957095809590959B01AC01BD01B6
:102F8000CF010895E199FECFBFBBAEBBE09A119689
:102F90000DB20895E199FECFBFBBAEBB0DBA11963D
:0C2FA0000FB6F894E29AE19A0FBE089573
:102FAC0001010200000A0000440000230023005429
:102FBC00646653636552620051610050600050605A
:102FCC00005161005262005363655464666768691E
:102FDC006A6B6B6A6968670000005353635353262E
:0C2FEC00034C026C030D0A0A1D000000DB
:00000001FF
